S01A000064656D6F70726F675F73746D3332673037312E7372656396
S3150800280000900020892F0008692F00086B2F000808
S3150800281000000000000000000000000000000000AA
S315080028200000000000000000000000006D2F0008F6
S3150800283000000000000000006F2F0008712F00083C
S31508002840D92F0008D92F0008D92F0008D92F00083A
S31508002850D92F0008D92F0008D92F0008D92F00082A
S31508002860D92F0008D92F0008D92F0008D92F00081A
S31508002870D92F0008D92F0008D92F0008D92F00080A
S31508002880D92F0008D92F0008D92F0008D92F0008FA
S31508002890D92F0008D92F0008D92F0008D92F0008EA
S315080028A0D92F0008D92F0008D92F0008D92F0008DA
S315080028B0D92F0008D92F0008D92F0008EE11AA55DC
S315080028C010B5064C2378002B07D1054B002B02D0F8
S315080028D0044800E000BF0123237010BD0C0000204F
S315080028E000000000A44C0008044B10B5002B03D0D0
S315080028F00349044800E000BF10BDC04600000000C0
S3150800290010000020A44C0008002243088B4274D310
S3150800291003098B425FD3030A8B4244D3030B8B42D2
S3150800292028D3030C8B420DD3FF22090212BA030CDB
S315080029308B4202D31212090265D0030B8B4219D3BC
S3150800294000E0090AC30B8B4201D3CB03C01A5241DC
S31508002950830B8B4201D38B03C01A5241430B8B4224
S3150800296001D34B03C01A5241030B8B4201D30B030D
S31508002970C01A5241C30A8B4201D3CB02C01A524134
S31508002980830A8B4201D38B02C01A5241430A8B42F7
S3150800299001D34B02C01A5241030A8B4201D30B02E0
S315080029A0C01A5241CDD2C3098B4201D3CB01C01AFA
S315080029B0524183098B4201D38B01C01A5241430904
S315080029C08B4201D34B01C01A524103098B4201D3F2
S315080029D00B01C01A5241C3088B4201D3CB00C01A5F
S315080029E0524183088B4201D38B00C01A52414308D7
S315080029F08B4201D34B00C01A5241411A00D20146FC
S31508002A00524110467047FFE701B5002000F006F86E
S31508002A1002BDC0460029F7D076E770477047C04622
S31508002A20002B11D1002A0FD1002900D1002802D08D
S31508002A300021C943081C07B4024802A140180290A5
S31508002A4003BDC046D9FFFFFF03B4684601B5029827
S31508002A5000F006F8019B9E4602B00CBC7047C046C3
S31508002A60F0B54F464646D646C0B5040082B00D00BE
S31508002A70914698468B422FD82CD04146484600F0BE
S31508002A80B1F829000600200000F0ACF8331A9C467D
S31508002A90203B9A4600D576E04B46524693401F00A7
S31508002AA04B46624693401E00AF4228D825D053466F
S31508002AB0A41BBD41002B00DA7BE000220023009214
S31508002AC001930123524693400193012362469340A2
S31508002AD0009318E08242D0D9002200230092019385
S31508002AE00A9B002B01D01C605D600098019902B01A
S31508002AF01CBC90469946A246F0BDA342D7D90022EF
S31508002B000023009201936346002BE9D0FB07984601
S31508002B10414672080A437B0866460EE0AB4201D17D
S31508002B20A2420CD8A41A9D41012024196D41002106
S31508002B30013E24184D41002E06D0AB42EED9013E87
S31508002B4024196D41002EF8D10098019953460019B1
S31508002B506941002B23DB2B005246D3402A006446EA
S31508002B60E2401C0053461500002B2DDB2600574675
S31508002B70BE40330026006746BE403200801A99419F
S31508002B8000900191ACE7624620239B1A4A46DA4038
S31508002B906146130042468A4017001F4380E7624693
S31508002BA020239B1A2A0066469A402300F3401343C3
S31508002BB0D4E76246202300219B1A00220091019245
S31508002BC00122DA40019280E72023624626009B1AFA
S31508002BD0DE402F00B0466646B74046463B003343C4
S31508002BE0C8E7C04610B5002903D100F007F8203021
S31508002BF002E0081C00F002F810BDC0461C210123A3
S31508002C001B04984201D3000C10391B0A984201D3C1
S31508002C10000A08391B09984201D30009043902A29F
S31508002C20105C40187047C046040302020101010106
S31508002C30000000000000000010B500F0C7F800F022
S31508002C4095F800F031F810BD10B500F097F800F0CF
S31508002C5089F810BD10B50A480A4B0360E1231B0228
S31508002C60436000238360C360036183610C22426171
S31508002C70C361802212010262436201F0AFFF10BDF8
S31508002C80280000200044004010B50100002301225E
S31508002C90044801F0BBFE002801D0002010BD013019
S31508002CA0FCE7C0462800002010B5FFF7D3FF10BD8B
S31508002CB0BFF34F8F034B044ADA60BFF34F8FC0460A
S31508002CC0FDE7C04600ED00E00400FA0510B5214B0B
S31508002CD01B78002B16D12048FFF7D6FF012800D015
S31508002CE010BD1D4B1B78013BDBB23F2BF8D800F01B
S31508002CF06EF81A4B1860174B01221A70184B0022EF
S31508002D001A70EDE7164B1B7801331348C018FFF706
S31508002D10BBFF012813D1124A13780133DBB21370B3
S31508002D200D4A12789342DBD10A4A002111700A4AE9
S31508002D305278FF2AD4D1022BD2D1FFF7B9FF00F07F
S31508002D4046F8064B1B6864339842C9D9014B0022E2
S31508002D501A70C5E7F5000020B4000020F80000202E
S31508002D60F600002010B5FFF7B1FF10BD10B5A02082
S31508002D7000222021C00500F097FA10BD10B500F01A
S31508002D8026F804000F4B1B68C31AF422FF3293423D
S31508002D900ED90D4B1B78002B0BD10B4BF33AFF3A90
S31508002DA01A70A0202021C00500F07EFA054B1C6091
S31508002DB010BD054B00221A70A0202021C00500F086
S31508002DC073FAF3E700010020FC000020704710B5F5
S31508002DD000F050F910BD0000014A024B9A60704796
S31508002DE00028000800ED00E030B587B01422002165
S31508002DF001A801F04FFF0E4B5A6B012422435A6378
S31508002E005B6B23400093009BA025ED050022202143
S31508002E10280000F049FA2023019302940023039323
S31508002E20049301A9280000F085F907B030BDC04613
S31508002E300010024030B5A1B03822002112A801F0D6
S31508002E4029FF102200210EA801F024FF34220021B8
S31508002E5001A801F01FFF8020800000F02BFA022451
S31508002E60129480235B00159300251695C03B179393
S31508002E7019941A9430221B921C9380239B021D934B
S31508002E8080239B041E93C023DB051F9312A800F022
S31508002E903BFA07230E930F941095119502210EA85D
S31508002EA000F0F0FC0194039501A800F0CBFD21B0D9
S31508002EB030BD10B5FFF790FF00F0BCF8FFF7BAFF7A
S31508002EC0FFF792FFFFF7B8FEFFF7BEFEFCE700002C
S31508002ED000B583B00B4B196C012211431964196CA8
S31508002EE00A400092009ADA6B802149050A43DA63A0
S31508002EF0DB6B0B400193019BC020C00000F0C0F8BB
S31508002F0003B000BD0010024010B588B004001422BA
S31508002F10002103A801F0BEFE2268114B9A4201D097
S31508002F2008B010BD0F4BD96B802080020143D963CE
S31508002F30DA6B02400192019A596B012211435963D7
S31508002F405B6B13400293029B0C2303930A3B049387
S31508002F500792A02003A9C00500F0ECF8E0E7C046F8
S31508002F6000440040001002407047FEE77047704773
S31508002F7010B500F073F810BD024B802212059A6056
S31508002F807047C04600ED00E00D488546002103E085
S31508002F900C4B5B58435004310B480C4B42189A4271
S31508002FA0F6D30B4A02E0002313600432094B9A4217
S31508002FB0F9D3FFF7E1FF01F049FEFFF77AFFFEE7D5
S31508002FC0009000202C4D0008000000200C00002076
S31508002FD00C00002008010020FEE7000010B50400E0
S31508002FE0114B1968002901D1012010BDFA20800073
S31508002FF0FFF78AFC01000D4B1868FFF785FC00F007
S315080030007DF800280DD1032C01D90120EDE7013008
S3150800301000222100404200F03FF8054B1C600020CA
S31508003020E3E70120E1E7C046040000200000002095
S315080030300800002010B5084A116880235B000B437E
S3150800304013600020FFF7CAFF041E02D001242000E7
S3150800305010BDFFF73DFFFAE700200240034A136858
S31508003060034909685B1813607047C04604010020CD
S3150800307004000020014B18687047C0460401002070
S31508003080034A136803490B40184310607047C0464B
S3150800309000000140FFF9FFFF70B5002811DB830827
S315080030A0144DC0339B005C5903221040C000FC320B
S315080030B016008640B44389010A40824022435A5189
S315080030C070BDC0B20F230340083B9B0806339B0024
S315080030D0094A944663445D6803242040C000FF22E1
S315080030E014008440A5438901114081402943596051
S315080030F0E6E7C04600E100E000ED00E001380A4BD3
S3150800310098420FD8094A50600948036A1B021B0AED
S31508003110C02109060B43036200239360073313603B
S31508003120002070470120FCE7FFFFFF0010E000E0E9
S3150800313000ED00E0F0B5C64600B500233BE00326E7
S3150800314000E00026AE4035003D43534E1834A40037
S31508003150A551802435594246D4432E0026404A6854
S31508003160D20302D5424615432E004B4D8027EE5119
S315080031708426AD592E0026404A68920302D5424657
S3150800318015432E00444D8427EE512D682E00264007
S315080031904A68D20202D5424615432E003E4D2E609D
S315080031A06D682C404A68920202D542462A431400AA
S315080031B0394A546001330A681400DC4069D0012595
S315080031C09D402A409046F5D04C68022C01D0122C1E
S315080031D00ED1DC080834A400275807261E40B6007E
S315080031E00F22B24097430A69B24016003E43265062
S315080031F002685F0003242600BE40F6433240944628
S315080032004A681440BC406246144304604C68621E17
S31508003210012A03D9112C01D0122C10D1846834400C
S31508003220A446CC68BC406246144384604468AC43F8
S315080032304A681209012515409D4025434560C46822
S3150800324026408C68BC403443C4604A68D200B1D575
S315080032509C0825001835AD000F4EAF5903251D40B3
S31508003260ED000F26AE40B743A026F605B04200D1C2
S3150800327067E70A4EB04208D0094EB04207D0094E59
S31508003280B04200D15BE705265CE701265AE702262D
S3150800329058E704BC9046F0BD0018024000040050F0
S315080032A000080050000C0050002A01D181627047C6
S315080032B08161FCE710B5104A136810490B400343B7
S315080032C0136080239B00984201D0002010BD0C4B50
S315080032D01A6853009B1858000A49FFF715FB013076
S315080032E0054B5B695B0503D5002803D00138F7E772
S315080032F00020EBE70320E9E700700040FFF9FFFF35
S315080033000000002040420F0070B582B0041E00D1B4
S315080033103EE20368DB0739D5C14A916838230B407A
S31508003320D16803220A40102B26D0082B26D06368C2
S315080033308022520293427FD0A022D202934200D129
S3150800334081E0B74B1A68B7490A401A601A68B64945
S315080033500A401A606368002B00D180E0FFF78AFEF6
S315080033600500AF4B1B689B0310D4FFF783FE401B79
S315080033706428F6D903200CE2032AD6D1A84B1B6889
S315080033809B0303D56368002B00D104E223689B07DF
S3150800339031D5A34A936838210B40D16803220A40E5
S315080033A0102B6AD0002B6BD19D4A1268520503D5A3
S315080033B0E268002A00D1F0E1994842689B490A4030
S315080033C0616909020A434260002B0DD103689849D6
S315080033D00B4021690B4303600368DB0A07221A4086
S315080033E0944BD340944A1360944B1868FFF7F6FD44
S315080033F0002800D0D3E123681B0700D481E0884B5E
S315080034009A6838231340182B73D0A369002B00D170
S3150800341091E0834A136E01210B431366FFF72AFED8
S3150800342005007F4B1B6E9B076BD4FFF723FE401BE3
S315080034300228F6D90320ACE1794A116880235B0299
S315080034400B43136086E7764B19688022D2020A433B
S315080034501A601968802252020A431A607AE7FFF74F
S3150800346009FE05006E4B1B689B038FD5FFF702FE0E
S31508003470401B6428F6D903208BE1022A92D193E7F0
S31508003480E368002B22D0664A136869490B40216914
S315080034900B431360116880235B000B431360FFF72F
S315080034A0E9FD05005E4B1B685B0506D4FFF7E2FDE8
S315080034B0401B0228F6D903206BE159494B685B4A41
S315080034C013406269120213434B6094E7544A136827
S315080034D05B490B401360FFF7CDFD0500504B1B6899
S315080034E05B0588D5FFF7C6FD401B0228F6D90320E1
S315080034F04FE14B4B1B6E9B0703D5A369002B00D1ED
S315080035004FE123685B0700D4A2E0454B9A6838234D
S315080035101340202B22D0424BDB6BDB0027D4404ADA
S31508003520D16B802040050143D163D36B03400193DF
S31508003530019B01251CE03A4A136E01218B43136651
S31508003540FFF798FD0500364B1B6E9B07D9D5FFF78D
S3150800355091FD401B0228F6D903201AE1304BDB6D9A
S315080035609B0775D5A368002B72D1012011E10025B0
S31508003570344B1B68DB051FD5A368012B30D0052B00
S3150800358034D0274BDA6D01218A43DA65DA6D0331C7
S315080035908A43DA65A368002B32D0FFF76BFD060075
S315080035A01F4BDB6D9B0751D4FFF764FD801B264B31
S315080035B09842F5D90320ECE0224A116880235B0083
S315080035C00B431360FFF756FD06001E4B1B68DB0511
S315080035D0D2D4FFF74FFD801B0228F6D90320D8E086
S315080035E00F4AD36D01210B43D365D3E70C4BDA6D34
S315080035F004210A43DA65DA6D03390A43DA65C9E74D
S31508003600FFF738FD0600064BDB6D9B071ED5FFF757
S3150800361031FD801B0C4B9842F5D90320B9E0C04612
S3150800362000100240FFFFFEFFFFFFFBFFFF80FFFFCA
S31508003630FFC7FFFF0024F400000000200800002058
S31508003640FFFEFFFF0070004088130000012D26D002
S31508003650E369002B00D1A6E0564A916838220A4051
S31508003660102A63D0022B20D0524B1A6852490A40BE
S315080036701A60DA6803218A43DA60DA684F490A4031
S31508003680DA60FFF7F7FC04004A4B1B689B014BD531
S31508003690FFF7F0FC001B0228F6D9032079E0454A1B
S315080036A0D36B47490B40D363D2E7424A1368424972
S315080036B00B401360FFF7DEFC05003E4B1B689B01C1
S315080036C006D5FFF7D7FC401B0228F6D9032060E091
S315080036D0384AD3683B491940236A606A0343A06A9B
S315080036E000020343E06A0343206B0343606B034312
S315080036F00B43D360116880235B040B431360D168C6
S3150800370080235B050B43D360FFF7B4FC0400294B09
S315080037101B689B0106D4FFF7ADFC001B0228F6D9EF
S31508003720032036E0002034E0002032E0012B3CD0B4
S31508003730204BDA6803231340216A8B4201D001200B
S3150800374027E070231340616A8B4201D0012020E0F4
S31508003750FE21C9011140A36A1B02994201D001202A
S3150800376017E0F8239B031340E16A8B4201D001203E
S315080037700FE0E0231B051340216B8B4201D001208B
S3150800378007E0520F5207636B9A4210D0012000E0FF
S31508003790012002B070BD0120FBE70120F9E70120F6
S315080037A0F7E70120F5E70020F3E70120F1E700201D
S315080037B0EFE7C04600100240FFFFFFFEFFFFFEEEE8
S315080037C0FFFFFFEF8C80C11110B52B4B9B68382289
S315080037D01A4219D0284B9A6838231340082B46D02A
S315080037E0254B9A6838231340102B18D0224B9A6819
S315080037F038231340202B3CD01F4B9A68382313409C
S31508003800182B31D0002009E01B4B1A68D20A07236F
S315080038101340012199401948FFF776F810BD164A5A
S31508003820D1680D3B0B40D2681209072111400131BE
S31508003830032B0FD11248FFF767F80F4BDA68120A05
S315080038407F23134058430C4BD968490F0131FFF7C2
S315080038505BF8E3E70948FFF757F8074BDA68120AF7
S315080038607F2313405843EEE7FA20C001D6E7044801
S31508003870D4E780200002D1E7001002400024F400BB
S3150800388000127A0070B504000D00002800D1AAE0E5
S31508003890574B1A68072313408B4221D323689A078C
S315080038A00ED55B0705D5534A9168E023DB010B4328
S315080038B09360504A936850490B40A1680B43936044
S315080038C02368DB0754D56368012B20D0022B3BD035
S315080038D0002B3FD1474A126852051CD401206AE0E2
S315080038E0434A136807218B432B431360FFF7C2FB38
S315080038F006003F4B1A6807231340AB42CED0FFF7AA
S31508003900B9FB801B3D4B9842F3D9032053E0394A53
S315080039101268920369D537498A6807208243134398
S315080039208B60FFF7A7FB0600324B9B6838221A40CC
S315080039306368DB009A421BD0FFF79CFB801B2F4B6A
S315080039409842F1D9032036E02A4A12689201E2D455
S31508003950012030E0032B05D0264AD26D9207DAD42F
S31508003960012028E0234A126E9207D4D4012022E0CF
S315080039701F4B1A6807231340AB421DD823685B0701
S3150800398006D51C4A93681E490B40E1680B439360B1
S31508003990FFF71AFF174B9A68120A0F2313409B006A
S315080039A0184A9A581F231340D840174B1860174BCC
S315080039B01868FFF713FB70BD0D4A136807218B4380
S315080039C02B431360FFF756FB0600094B1A680723BB
S315080039D01340AB42D2D0FFF74DFB801B074B9842F2
S315080039E0F3D90320E7E70120E5E70120E3E7C0462E
S315080039F00020024000100240FFF0FFFF881300007D
S31508003A00FF8FFFFFBC4C00080000002008000020C4
S31508003A10014B18687047C0460000002010B5FFF734
S31508003A20F7FF064B9A68120B072313409B00044ABC
S31508003A309A581F231340D84010BDC04600100240B4
S31508003A40FC4C0008F0B583B0040003689B0360D5FE
S31508003A50804BDB6BDB001ED47E4AD16B8020400591
S31508003A600143D163D36B03400193019B01267A4A34
S31508003A70116880235B000B431360FFF7FBFA050010
S31508003A80754B1B68DB0508D4FFF7F4FA401B0228C0
S31508003A90F6D9032502E00026E9E70025002D21D105
S31508003AA06C4BDB6DC0229200134010D0226B9A42F9
S31508003AB00DD0684AD36D69490B40D06D8021490203
S31508003AC00143D165D16D66480140D165D365DB07F1
S31508003AD010D4002D06D15F4AD36D60490B40216B87
S31508003AE00B43D365012E15D15A4AD36B5D490B405A
S31508003AF0D3630FE0FFF7BEFA0700564BDB6D9B0753
S31508003B00E7D4FFF7B7FAC01B574B9842F5D90325F8
S31508003B10DFE700252368DB0706D54E4A536D0321E8
S31508003B208B4361680B43536523689B0706D5494A4F
S31508003B30536D0C218B43A1680B43536523689B0681
S31508003B4006D5444A536D49490B40E1680B43536512
S31508003B5023689B0506D53F4A536D45490B40A16925
S31508003B600B43536523685B0506D53A4A536D4149AD
S31508003B700B40E1690B43536523685B0606D5354A56
S31508003B80536D3D490B4021690B43536523685B041C
S31508003B900BD5304A536D9B009B08216A0B4353652E
S31508003BA08023DB05226A9A4239D023681B0306D58F
S31508003BB0284A536D40218B43616A0B43536523683A
S31508003BC09B020BD5234A536D2C490B40A16A0B4324
S31508003BD053658023DB03A26A9A4227D023685B02D7
S31508003BE00BD51C4A536D26490B40E16A0B435365B6
S31508003BF080235B04E26A9A421FD023681B050BD513
S31508003C00144A536D1F490B4061690B43536562693A
S31508003C108023DB019A4215D0280003B0F0BD0D4A77
S31508003C20D16880235B020B43D360BEE7094AD1689B
S31508003C3080235B040B43D360D0E7064AD1680B4365
S31508003C40D360DAE7034AD16880235B020B43D3606B
S31508003C50E2E7C0460010024000700040FFFCFFFF8C
S31508003C60FFFFFEFFFFFFFFEF88130000FFF3FFFFD4
S31508003C70FFFFF3FFFFFFCFFFFFCFFFFFFFFFBFFFF2
S31508003C80FFFFFFFEFF3FFFFFF8B5040001688368EA
S31508003C900269134342691343C2691343426E1A43C6
S31508003CA00B68BD48034013430B6022685368BB4941
S31508003CB00B40E1680B435360A1692268B84B9A42EE
S31508003CC001D0236A19439368B64803400B439360AF
S31508003CD02268D36A0F218B43616A0B43D362236838
S31508003CE0B14A93425CD0B14A93426DD0B04A9342EE
S31508003CF000D19EE0AF4A934200D19CE0A84A934285
S31508003D0077D01025A64A934200D198E080231B025B
S31508003D10E2699A4200D151E3022D01D100F0F8FC84
S31508003D2001D800F0A1FC042D01D100F02DFD082DCD
S31508003D3001D000F093FD636A002B01D100F067FD06
S31508003D40012B01D100F06FFD022B01D100F06EFDB1
S31508003D50032B01D100F06DFD042B01D100F06BFDA2
S31508003D60052B01D100F06AFD062B01D100F068FD94
S31508003D70072B01D100F066FD082B01D100F065FD87
S31508003D80092B01D100F064FD0A2B01D100F063FD77
S31508003D900B2B01D100F039FD80231B0200F039FD01
S31508003DA0854A516D03220A40012A09D0002A05D006
S31508003DB0022A3AD0032A05D01025A3E70025A1E751
S31508003DC004259FE708259DE77B4A516D0C220A408A
S31508003DD0042A0AD005D9082A29D00C2A07D1082589
S31508003DE090E7002A03D100258CE704258AE71025E9
S31508003DF088E7714A526DC02109010A408021C9002D
S31508003E008A420ED009D9802109018A4215D0C021DB
S31508003E1009018A4207D1082574E7002A03D100253B
S31508003E2070E704256EE710256CE702256AE7022588
S31508003E3068E7002566E7002564E7022562E7022DA4
S31508003E4000D1C1E02ED9042D00D1DAE0082D01D029
S31508003E5000F007FD636A002B00D122E1012B00D197
S31508003E6022E1022B00D122E1032B00D122E1042B0F
S31508003E7000D121E1052B00D121E1062B00D120E15B
S31508003E80072B00D11FE1082B00D11FE1092B00D118
S31508003E901FE10A2B00D11FE10B2B00D1E9E080209E
S31508003EA0000226E0002D01D000F0DBFCFFF7B6FD8E
S31508003EB0636A002B1AD0012B5FD0022B5FD0032B2D
S31508003EC05FD0042B5FD0052B5FD0062B5FD0072B66
S31508003ED05FD0082B72D0092B72D00A2B72D00B2B0D
S31508003EE001D0012103E08021490000E00121FEF70D
S31508003EF00BFD002801D100F0B6FC626853009B1840
S31508003F00834201D900F0B1FC1303834201D200F0C9
S31508003F10AEFC022D00D142E100D8E0E0042D00D12C
S31508003F2086E1082D00D046E2636A002B00D110E234
S31508003F30012B00D11AE2022B00D11BE2032B00D180
S31508003F401CE2042B00D11CE2052B00D11DE2062B36
S31508003F5000D11DE2072B00D11DE2082B00D11EE27D
S31508003F60092B00D11FE20A2B00D120E20B2B00D12E
S31508003F70EBE1802636040027EEE10221B7E70421AB
S31508003F80B5E70621B3E70821B1E70A21AFE70C2117
S31508003F90ADE71021ABE7C046F369FFCFFFCFFFFFC0
S31508003FA000800040FFF4FF11003801400044004043
S31508003FB000480040004C004000100240202196E7CF
S31508003FC0402194E7802192E7636A002B53D0012BA6
S31508003FD053D0022B53D0032B53D0042B53D0052B8D
S31508003FE053D0062B53D0072B53D0082B53D0092B6D
S31508003FF053D00A2B53D00B2B01D0AA4879E7AA48ED
S3150800400077E7FFF7E1FB636A002B1AD0012B1CD078
S31508004010022B1CD0032B1CD0042B1CD0052B1CD028
S31508004020062B1CD0072B1CD0082B1CD0092B1CD008
S315080040300A2B1CD00B2B01D0012103E0802149005B
S3150800404000E00121FEF760FC53E70221FAE70421AC
S31508004050F8E70621F6E70821F4E70A21F2E70C213A
S31508004060F0E71021EEE72021ECE74021EAE780217E
S31508004070E8E780203DE78B483BE78C4839E78C48E2
S3150800408037E78C4835E78C4833E78C4831E78C4866
S315080040902FE78C482DE78C482BE78C4829E78C4876
S315080040A027E78020000224E78020C00121E780203E
S315080040B080011EE787481CE78020400119E78648EB
S315080040C017E7864815E78020000112E78020C00020
S315080040D00FE7802080000CE78020400009E7002DCC
S315080040E000D068E1FFF79AFC636A002B1CD0012B0D
S315080040F037D0022B38D0032B39D0042B3AD0052BD6
S315080041003BD0062B3CD0072B3DD0082B3ED0092BA5
S315080041103FD00A2B40D00B2B02D00122002305E00A
S3150800412080225200002301E0012200230021FEF72D
S3150800413077FC050E0B022B4302026568680800210E
S31508004140801859412A000023FEF76AFC0200002065
S315080041506349644BD3188B4200D98AE32368DA6033
S31508004160B9E202220023E1E704220023DEE7062261
S315080041700023DBE708220023D8E70A220023D5E735
S315080041800C220023D2E710220023CFE720220023A7
S31508004190CCE740220023C9E780220023C6E7636AEA
S315080041A0002B1BD0012B25D0022B26D0032B27D082
S315080041B0042B28D0052B29D0062B2AD0072B2BD049
S315080041C0082B2CD0092B2DD00A2B2ED00B2B02D046
S315080041D0454E002704E0334E002701E0424E0027F3
S315080041E050080021801979410023FEF719FC0200C6
S315080041F00020ADE73D4E0027F2E73D4E0027EFE7EA
S315080042003C4E0027ECE73C4E0027E9E73B4E0027EB
S31508004210E6E73B4E0027E3E73A4E0027E0E73A4E4B
S315080042200027DDE7394E0027DAE7394E0027D7E7BA
S31508004230FFF7CAFA636A002B1CD0012B2FD0022B7A
S3150800424068D0032B69D0042B6AD0052B6BD0062BBC
S315080042506CD0072B6DD0082B6ED0092B6FD00A2B8C
S3150800426070D00B2B02D00122002305E080225200D9
S31508004270002301E0012200230021FEF7D1FB050EF1
S315080042800B022B4302026568680800218018594111
S315080042902A000023FEF7C4FB0200002058E702228A
S315080042A00023E9E70024F40024F4000000127A0051
S315080042B000093D00AAB0280080841E00006A180084
S315080042C05558140040420F0020A1070090D0030063
S315080042D048E8010055150000CC0C0000AA0A0000A9
S315080042E0FFFC0F0000FDFFFF000024F40000127A17
S315080042F00000093D00AAB0280080841E00006A1844
S31508004300005558140040420F0020A1070090D00322
S315080043100048E80104220023AEE706220023ABE7A3
S3150800432008220023A8E70A220023A5E70C22002377
S31508004330A2E7102200239FE7202200239CE74022C1
S31508004340002399E78022002396E780263602002775
S3150800435002E080263604002750080021801979419A
S315080043600023FEF75DFB02000020F1E68026F60337
S315080043700027F1E78026B6030027EDE7A74E0027BA
S31508004380EAE7802676030027E6E7A54E0027E3E757
S31508004390A44E0027E0E7802636030027DCE78026C0
S315080043A0F6020027D8E78026B6020027D4E780263B
S315080043B076020027D0E701200022C9E6022D00D1A7
S315080043C082E02DD9042D00D1BAE0082D00D022E1D3
S315080043D0636A002B00D1F7E0012B00D100E1022B24
S315080043E000D100E1032B00D100E1042B00D1FFE04E
S315080043F0052B00D1FFE0062B00D1FEE0072B00D1EC
S31508004400FDE0082B00D1FDE0092B00D1FDE00A2BC9
S3150800441000D1FDE00B2B00D1D4E080235B02D5E070
S31508004420002D00D0F7E0FFF7F9FA636A002B1AD0DF
S31508004430012B35D0022B35D0032B35D0042B35D0A4
S31508004440052B35D0062B35D0072B35D0082B35D084
S31508004450092B35D00A2B35D00B2B01D0012103E0CF
S315080044608021490000E00121FEF74EFA400063680A
S315080044705B08C0186168FEF747FA03041B0C0020A6
S3150800448069491A00103A8A4200D9F4E10F22190044
S3150800449091435B08083A13400B432268D3601AE13C
S315080044A00221E1E70421DFE70621DDE70821DBE752
S315080044B00A21D9E70C21D7E71021D5E72021D3E730
S315080044C04021D1E78021CFE7636A002B19D0012B61
S315080044D022D0022B22D0032B22D0042B22D0052B4C
S315080044E022D0062B22D0072B22D0082B22D0092B2C
S315080044F022D00A2B22D00B2B01D04C4B02E04C4B7E
S3150800450000E04A4B62685008C0181100FEF7FCF933
S3150800451003041B0C0020B3E7464BF3E7464BF1E7D1
S31508004520464BEFE7464BEDE7464BEBE7464BE9E7ED
S31508004530464BE7E7464BE5E7464BE3E7464BE1E7FD
S31508004540FFF742F9636A002B1AD0012B26D0022BFB
S3150800455026D0032B26D0042B26D0052B26D0062BB7
S3150800456026D0072B26D0082B26D0092B26D00A2B97
S3150800457026D00B2B01D0012103E08021490000E061
S315080045800121FEF7C1F9400063685B08C01861683D
S31508004590FEF7BAF903041B0C002071E70221F0E7C5
S315080045A00421EEE70621ECE70821EAE70A21E8E715
S315080045B00C21E6E71021E4E72021E2E74021E0E7C5
S315080045C08021DEE7F53301E080235B02626850084C
S315080045D0C0181100FEF798F903041B0C00204FE7DA
S315080045E080231B02F2E78023DB01EFE71B4BEDE795
S315080045F080239B01EAE71A4BE8E71A4BE6E7802394
S315080046005B01E3E780231B01E0E78023DB00DDE7AE
S3150800461080239B00DAE70120002331E700551500C7
S3150800462000CC0C0000AA0A00EFFF00000048E801D1
S3150800463048E801000024F40000127A005461510091
S3150800464000093D0000D43000AAB0280080841E006E
S3150800465040420F0020A1070090D00300AA2A0000BC
S315080046609819000054150000002D00D0F6E0FFF759
S31508004670D5F9636A002B1AD0012B35D0022B35D019
S31508004680032B35D0042B35D0052B35D0062B35D04A
S31508004690072B35D0082B35D0092B35D00A2B35D02A
S315080046A00B2B01D0012103E08021490000E0012104
S315080046B0FEF72AF963685B08C0186168FEF724F9F3
S315080046C003041B0C00206E491A00103A8A4200D9CE
S315080046D0D3E02268D36001236A22A352023AA35286
S315080046E00023E3662367F8BD0221E1E70421DFE73B
S315080046F00621DDE70821DBE70A21D9E70C21D7E700
S315080047001021D5E72021D3E74021D1E78021CFE743
S31508004710636A002B19D0012B22D0022B22D0032B3F
S3150800472022D0042B22D0052B22D0062B22D0072BF1
S3150800473022D0082B22D0092B22D00A2B22D00B2BD1
S3150800474001D0504B02E0504B00E04E4B62685008D7
S31508004750C0181100FEF7D8F803041B0C0020B2E7B6
S315080047604A4BF3E74A4BF1E74A4BEFE74A4BEDE78B
S315080047704A4BEBE74A4BE9E74A4BE7E74A4BE5E79B
S315080047804A4BE3E74A4BE1E7FFF71EF8636A002B5B
S315080047901AD0012B25D0022B25D0032B25D0042B8C
S315080047A025D0052B25D0062B25D0072B25D0082B61
S315080047B025D0092B25D00A2B25D00B2B01D001217A
S315080047C003E08021490000E00121FEF79DF86368B7
S315080047D05B08C0186168FEF797F803041B0C0020F5
S315080047E071E70221F1E70421EFE70621EDE7082149
S315080047F0EBE70A21E9E70C21E7E71021E5E72021A5
S31508004800E3E74021E1E78021DFE7753301E0802314
S315080048101B0262685008C0181100FEF775F80304F9
S315080048201B0C00204FE78023DB01F2E780239B0166
S31508004830EFE7204BEDE780235B01EAE71E4BE8E74D
S315080048401E4BE6E780231B01E3E78023DB00E0E756
S3150800485080239B00DDE780235B00DAE70120002345
S3150800486031E7012037E7002035E7012033E701204B
S3150800487031E701202FE701202DE701202BE7C0466D
S31508004880EFFF00000024F40024F4000000127A0070
S3150800489000093D00AAB0280080841E00006A18009E
S315080048A05558140040420F0020A1070090D003007D
S315080048B048E8010055150000CC0C0000AA0A0000C3
S315080048C0836ADB0706D5026853682C490B40C16A20
S315080048D00B435360836A9B0706D5026853682849C9
S315080048E00B40016B0B435360836A5B0706D502686E
S315080048F0536824490B40416B0B435360836A1B077B
S3150800490006D50268536820490B40816B0B435360F8
S31508004910836ADB0606D5026893681C490B40C16B9F
S315080049200B439360836A9B0606D502689368184909
S315080049300B40016C0B439360836A5B060BD50268D8
S31508004940536814490B40416C0B43536080235B0347
S31508004950426C9A420AD0836A1B0606D502685368D7
S315080049600D490B40C16C0B4353607047026853688E
S315080049700A490B40816C0B435360ECE7FFFFFDFFD0
S31508004980FFFFFEFFFFFFFBFFFF7FFFFFFFEFFFFFBE
S31508004990FFDFFFFFFFFFEFFFFFFFF7FFFFFF9FFFB1
S315080049A0F0B5C64600B506000C0017009846069DE9
S315080049B03368DB6923401B1B5A425341BB421ED155
S315080049C06B1CF5D0FEF756FB4346C01AA84201D821
S315080049D0002DEDD1326813680B490B40136032681D
S315080049E09368A331FF318B43936020238022B35011
S315080049F00432B3505C330022F254032000E0002056
S31508004A0004BC9046F0BDC0465FFEFFFFF0B5C64643
S31508004A1000B584B004000F0016001D008423C35897
S31508004A20202B00D093E0002900D195E0002A00D180
S31508004A3094E080235B0182689A4222D07C23E35C5F
S31508004A40012B00D18CE07C230122E2540C33002296
S31508004A50E250043B2232E250FEF70CFB03905C2343
S31508004A60E6520233E652A3688022520193420FD0DF
S31508004A70002B1CD12269002A15D16032FF21A152D0
S31508004A801CE00369002BD9D1CB07D7D501205FE0FD
S31508004A902269002A03D160323349A1520EE060220E
S31508004AA0FF21A1520AE060227F21A15206E080225E
S31508004AB0520593420BD060220021A1526022A65AC9
S31508004AC08022520193420DD00023984620E02269A5
S31508004AD0002A03D160327F21A152EFE760223F21ED
S31508004AE0A152EBE72369002B02D0002398460FE07A
S31508004AF0B84600270CE023685B6A334042461380B9
S31508004B0002239C46E0445E22A35A013B9BB2A35271
S31508004B105E23E35A9BB2002B11D00095039B00221B
S31508004B2020212000FFF73CFF00281BD1002FE2D0F0
S31508004B3023685B6AF2B213403B700137E3E78433BC
S31508004B402022E250083B0022E254002000E0022026
S31508004B5004B004BC9046F0BD0120F9E70120F7E750
S31508004B600220F5E70320F3E7FF01000030B583B024
S31508004B70040088230022C250FEF77CFA0500236849
S31508004B801B681B070ED423681B685B0717D42023F2
S31508004B908022A3500432A3505C330022E254002042
S31508004BA003B030BD80210C4B00930300002289031B
S31508004BB02000FFF7F5FE0028E5D00320F0E7802166
S31508004BC0054B00932B000022C9032000FFF7E8FEDF
S31508004BD00028DCD00320E3E7FFFFFF0110B5041E21
S31508004BE030D08023C358002B22D080232422E250C1
S31508004BF02268136801218B4313602000FFF744F8ED
S31508004C00012814D0A36A002B18D1226853680E49CC
S31508004C100B405360226893682A218B43936022686D
S31508004C20136829390B4313602000FFF79FFF10BD57
S31508004C307C330022C254FEF767F9D6E72000FFF757
S31508004C403FFEE2E70120F2E7FFB7FFFF70B5002657
S31508004C500C4D0D4C641BA410A64209D1002600F089
S31508004C6021F80A4D0A4C641BA410A64205D170BD52
S31508004C70B300EB5898470136EEE7B300EB58984770
S31508004C800136F2E7244D0008244D0008244D00089B
S31508004C90284D000803001218934200D17047197076
S31508004CA00133F9E7F8B5C046F8BC08BC9E4670471C
S31108004CB0F8B5C046F8BC08BC9E46704724
S31508004CBC00000000000000000000000000000000DA
S31508004CCC00000000000000000000000000000000CA
S31508004CDC01000000020000000300000004000000B0
S31508004CEC060000000700000008000000090000008C
S31508004CFC000000000000000000000000000000009A
S31508004D0C010000000200000003000000040000007F
S30D08004D1C44DDFF7F01000000E1
S30908004D24E928000864
S30908004D28C128000888
S31108004D2C0024F400010000000400000050
S70508002F893A
